:020000009C283A
:080008008C0003088D00910A31
:10001000031D0C280E179103743081000B110D087D
:1000200083008C0E0C0E09008A0114083F398207E8
:100030002034653461346934773472347534733400
:100040006A3470345F346C345F34663476346834C8
:1000500031345F345F345F345F347C345F345F3419
:1000600032345F345F345F343334213434343534E4
:100070005F3427345F345F345F345F345F345F3420
:100080005F345F342E345F345F3422345F345F3446
:100090005F345F345F343F345F345F345F345F34E8
:1000A0005F345F343C345F345F345F345F345F34DB
:1000B0008A0114083F398207203474346E346D3459
:1000C00064346B3467346F34623478346334793435
:1000D0007A3471345F345F3436343D342F345F34D6
:1000E0005F343E3428345F3437345F345F345F34F8
:1000F00038345F34393430345F342D345F345F3416
:100100005F345F345F345F345F345F343B345F347B
:100110005F3429345F345F345F345F345F342C34B0
:100120005F345F345F345F343A345F345F345F345C
:100130005F345F345F345F34043062000F30650039
:1001400005128F30660090018F018F0BA528900B50
:10015000A5285821223086004A21203086004A21D5
:100160000C304A2106304A2127304A210D309500B3
:1001700015308400840A8001950BBA28183093004A
:1001800081018E018B018B168B17861FC5280516E2
:10019000861BC8280512910102301102031CCC28CD
:1001A000861FD02811089200910105160130940095
:1001B000130812020318DF288E171E21E1288E1360
:1001C0002F21861BE12811089200910105121308C6
:1001D0001202031CF128EC28130D1202031C0E2935
:1001E000152902301102031CF228861FF528110878
:1001F000920091010516130812020318072900291D
:100200001E218E1B03148E1F0310940DE1282F2135
:100210008E1F03148E1B0310940DE1288E1B1229D0
:100220005820132914204721CC288E1B1C29582024
:10023000472120304721CC28142018291508183EC2
:10024000840000089602120880009607160C97009A
:10025000970C3F309705950A033095053F291C08F8
:100260001F3E840000089D02120880009D071D0C9F
:100270009E009E0C3F309E059C0A03309C0517088B
:100280001E0293000310930C1708930708008601C1
:1002900006174B2986019000100E0F3986040616AA
:1002A0000612F030860510080F398604061606126D
:1002B0008F306600A03086000616060890000612F1
:0E02C0000616061290195A29803066000800B2
:02400E00F23F7F
:00000001FF
